:100000000AC023C022C021C020C01FC01EC01DC006
:100010001CC01BC01AC011241FBECFEDCDBF10E005
:10002000A0E6B0E0ECE1F1E003C0C89531960D9296
:10003000A036B107D1F710E0A0E6B0E001C01D92F4
:10004000A036B107E1F72CD068C0DACF80E888BBD2
:1000500087BB12BA82E081BB0895262F372F482F25
:10006000592F84E0220F331F441F551F8A95D1F763
:1000700060E876E988E990E029D02150304029B93C
:100080008AB188618AB908955D9BFECF8CB90895C5
:100090005F9903C080E090E008958CB1992708959E
:1000A00080E888BB87BB12BA82E081BB60E875E25A
:1000B00080E090E0D2DF5F9BFECF8CB19927282FA4
:1000C0008823C9F35D9BFECF2CB9F5CFA1E21A2E90
:1000D000AA1BBB1BEA2FFB2F0DC0AA1FBB1FEE1FC5
:1000E000FF1FA217B307E407F50720F0A21BB30B0D
:1000F000E40BF50B661F771F881F991F1A9469F789
:100100006095709580959095262F372F482F592F01
:0C0110006A2F7B2F8E2F9F2F0895FFCFAA
:00000001FF
